S026000062696E2F6F70656E626C745F6E75636C656F5F73746D33326631303372622E73726563D7
S315080000000050002075020008BD020008BD02000865
S31508000010BD020008BD020008BD020008000000007D
S31508000020000000000000000000000000BD020008FB
S31508000030BD02000800000000BD02000811130008F8
S31508000040BD020008BD020008BD020008BD02000886
S31508000050BD020008BD020008BD020008BD02000876
S31508000060BD020008BD020008BD020008BD02000866
S31508000070BD020008BD020008BD020008BD02000856
S31508000080BD020008BD020008BD020008BD02000846
S31508000090BD020008BD020008BD020008BD02000836
S315080000A0BD020008BD020008BD020008BD02000826
S315080000B0BD020008BD020008BD020008BD02000816
S315080000C0BD020008BD020008BD020008BD02000806
S315080000D0BD020008BD020008BD020008BD020008F6
S315080000E0BD020008BD020008BD02000800000000AD
S315080000F000000000000000000000000000000000F2
S3110800010000000000000000005FF808F195
S3150800010C10B5054C237833B9044B13B10448AFF337
S3150800011C00800123237010BD40040020000000005D
S3150800012C6418000808B5034B1BB103490348AFF321
S3150800013C008008BD00000000440400206418000874
S3150800014C70B50D4E0D4D761BB61006D00024013435
S3150800015C55F8043B9847A642F9D1094E094D01F0CA
S3150800016C7BFB761BB61006D00024013455F8043BED
S3150800017C9847A642F9D170BDD0180008D0180008C7
S3150800018CD8180008D0180008024B13B1024800F022
S3150800019C05B8704700000000B501000800230146A9
S315080001AC1A46184600F01EB838B50A4C0A4D641B98
S315080001BCA4100AD004F18043013B05EB8305013CEE
S315080001CC55F804399847002CF9D1BDE8384001F0A8
S315080001DC49BB00BFDC180008D8180008704700BFD8
S315080001EC704700BF2DE9F0411D4C05462068904626
S315080001FC1F460E46FFF7F2FF1A4B1A68D2F848311B
S3150800020C1BB35A6820681F2A24DC4DB9511C0232CC
S3150800021C596043F82260FFF7E3FF0020BDE8F08140
S3150800022C012403EB820CCCF88880D3F8881194400F
S3150800023C2143022DC3F88811CCF80871E6D1D3F8FE
S3150800024C8C110C43C3F88C41E0E702F5A673C2F88F
S3150800025C4831D6E7FFF7C4FF4FF0FF30DEE700BFA3
S3150800026C280400207C180008002103E00B4B5B587F
S3150800027C435004310A480B4B42189A42F6D30A4AA1
S3150800028C02E0002342F8043B084B9A42F9D300F0EB
S3150800029CE3FBFFF755FF00F0AFFC7047DC180008CE
S315080002AC000000203C04002040040020980900208F
S315080002BCFEE70000014B1860704700BF34040020AD
S315080002CCC36813F4005F01D00120704730B585B0C0
S315080002DC0D460446C36823F4B05323F00C034A684E
S315080002ECC9680A4329690A431343C360AB680269A0
S315080002FC22F44052134303616B69426922F440723B
S3150800030C13434361684600F06BF91C4B9C4208D0BA
S3150800031C1B4B9C422AD01B4B9C4229D0012005B072
S3150800032C30BD039B33B32A6832B303EB830303EB69
S3150800033C83039200B3FBF2F3134DA5FB032040098C
S3150800034C020191B2642202FB103213013233A5FB6F
S3150800035C0323C3F34F1303F0F0020A4492B203F0DB
S3150800036C0F0313449BB2A3600020D8E7029BD9E77E
S3150800037C029BD7E70120D2E70120D0E700380140DD
S3150800038C00440040004800401F85EB51074AD368DB
S3150800039C23F4E0631B041B0C000200F4E060184312
S315080003AC40F0BF6040F40030D060704700ED00E0CC
S315080003BC30B4174BDB68C3F30223C3F10704042CD0
S315080003CC28BF04241D1D062D01D9033B00E000237C
S315080003DC4FF0FF3505FA04F421EA0401994005FAB1
S315080003EC03F322EA03031943002809DB0901C9B2FE
S315080003FC00F1604000F5614080F8001330BC70478E
S3150800040C00F00F000901C9B2024B1954F6E700BFF8
S3150800041C00ED00E014ED00E00138B0F1807F0AD25F
S3150800042C064B5860064AF02182F823100020986083
S3150800043C07221A6070470120704700BF10E000E0E1
S3150800044C00ED00E010B5064B4FF0FF32DA600024E1
S3150800045C1C61DA60DC6000F03DFC204610BD00BF74
S3150800046C0010024010B504460E4B18784FF47A73F8
S3150800047CB3FBF0F30C4A1068B0FBF3F0FFF7CCFFB4
S3150800048C68B90F2C01D901200AE0002221464FF049
S3150800049CFF30FFF78DFF054B1C60002000E00120A4
S315080004AC10BD00BF2C0400203404002030040020AA
S315080004BC08B5074A136843F0100313600320FFF7C7
S315080004CC65FF0020FFF7CEFF00F09EFB002008BD5D
S315080004DC00200240184A136843F001031360164BB8
S315080004EC1B6813F0020FFAD0134A536823F0030360
S315080004FC5360114B5B6813F00C0FFAD10E4A136854
S3150800050C23F0807313600C4B1B6813F0007FFAD131
S3150800051C094B002058601A6822F450221A601A688F
S3150800052C22F0F80242F080021A6098605A6A42F089
S3150800053C80725A62704700BF00100240034B5B681A
S3150800054CC3F30313024AD35CD84070470010024029
S3150800055C80180008034B5B68C3F30223024AD35C7A
S3150800056CD84070470010024090180008034B5B688F
S3150800057CC3F3C223024AD35CD8407047001002402A
S3150800058C901800080B4B5B6803F4803343B90A4890
S3150800059C084B5B68C3F38343023300FB03F07047D5
S315080005AC044B5868C0F34040431C0448B0FBF3F0B6
S315080005BCEEE700BF0010024000093D0000127A0069
S315080005CC08B5054B5B6803F00C03082B01D00348F0
S315080005DC08BDFFF7D7FFFBE70010024000127A00B0
S315080005EC10B50446FFF7ECFF2060FFF7A7FF606025
S315080005FCFFF7B0FFA0606068FFF7B8FFE06010BDBA
S3150800060C264B98420DD0264B984216D0254B98422D
S3150800061C1FD0254B984228D0244B984231D0012024
S3150800062C704703F58433DA6842F00402DA60DA6854
S3150800063C22F00402DA600020704703F58233DA6888
S3150800064C42F00802DA60DA6822F00802DA60002062
S3150800065C704703F58033DA6842F01002DA60DA681C
S3150800066C22F01002DA600020704703F57C43DA6842
S3150800067C42F02002DA60DA6822F02002DA60002002
S3150800068C704703F57843DA6842F04002DA60DA68B4
S3150800069C22F04002DA600020704700BF00080140D3
S315080006AC000C0140001001400014014000180140E4
S315080006BCF0B50D68C5F30F2595FAA5F2B2FA82F2D4
S315080006CC35E0A2F108044FF00113A34043F0806310
S315080006DC39E0C45993FAA3F6B6FA86F6B6004FF083
S315080006EC030C0CFA06F624EA060C93FAA3F6B6FAE9
S315080006FC86F6B6008C6804FA06F646EA0C06C65167
S3150800070CCC6893FAA3FCBCFA8CFC4FEA8C0C4FF021
S3150800071C040E0EFA0CFC26EA0C0693FAA3F3B3FAAB
S3150800072C83F39B0004FA03F33343C351013235FABE
S3150800073C02F335D0012393402B42F7D0072AC0D8B1
S3150800074C40F2011393404E681F0EC45993FAA3FC4A
S3150800075CBCFA8CFC4FEA8C0C4FF00F0E0EFA0CFC04
S3150800076C24EA0C0493FAA3FCBCFA8CFC4FEA8C0C16
S3150800077C06FA0CF63443C451C6681C0A26EA040C5D
S3150800078C94FAA4F4B4FA84F40E6906FA04F44CEA5E
S3150800079C0404C4604C68012C9BD0092CC6D198E77C
S315080007AC0020F0BD044B0022DA61044A136943F0B9
S315080007BC010313610180704778090020002002406C
S315080007CC154BDB6813F0100F06D0144AD36943F0A7
S315080007DC0203D361102300E000230F4AD26812F0FB
S315080007EC040F06D00D49CA6942F00102CA6143F0EA
S315080007FC0403094AD26912F0010F09D00749CA69DC
S3150800080C42F00402CA610449CA6922F00102CA61AB
S3150800081C014AD360704700BF0020024078090020C7
S3150800082C0A4B1B6913F0800F0BD0084B084A5A6009
S3150800083C02F188325A601B6913F0800F03D100202D
S3150800084C7047002070470120704700BF0020024007
S3150800085C23016745034A136943F08003136100209B
S3150800086C704700BF0020024038B5044600F046FD2C
S3150800087C0546164BDB6813F0010F0AD0B4F1FF3F9F
S3150800088CF7D024B100F03AFD401BA042F1D9032061
S3150800089C1BE00E4BDB6813F0200F02D00B4B20220B
S315080008ACDA600A4BDB6813F0100F0BD1074BDB69C8
S315080008BC13F0010F06D1054BDB6813F0040F01D1B9
S315080008CC002002E0FFF77CFF012038BD0020024023
S315080008DC2DE9F843234C247E012C41D01E46904624
S315080008EC0F4604461F4B01221A764CF25030FFF77E
S315080008FCBBFF034670BB012C29D0022C24D04FF029
S3150800090C040900244C4525D22101C1F12002A1F18C
S3150800091C200328FA01F106FA02F2114326FA03F328
S3150800092C194389B207EB4400FFF73CFF4CF25030F1
S3150800093CFFF79AFF0C4B1D6925F001051D6103464F
S3150800094C40B90134E4B2DDE74FF00209D9E74FF0BC
S3150800095C0109D6E7034A002111761846BDE8F88343
S3150800096C0223FAE77809002000200240064B0022F1
S3150800097CDA61064B1A6942F004021A611A6942F0E6
S3150800098C40021A61704700BF780900200020024017
S3150800099C064B0022DA61064B1A6942F002021A610A
S315080009AC58611A6942F040021A61704778090020AA
S315080009BC00200240264B1B7E012B46D070B50E46F6
S315080009CC0546234B01221A760368022B20D04CF2DB
S315080009DC5030FFF749FF90BB4FF0FF333360AC68DC
S315080009EC0121EA68AB6803EB8223A34228D9204687
S315080009FCFFF7CEFF4CF25030FFF736FF154A136956
S31508000A0C23F0020313610146B8B904F58064E8E7DC
S31508000A1C4CF25030FFF728FF08B1012110E00120F5
S31508000A2CFFF7A4FF4CF25030FFF71EFF0146094AA8
S31508000A3C136923F00403136102E0346000E001211A
S31508000A4C034B00221A76084670BD022108467047E9
S31508000A5C78090020002002400F4B1A6842F0010268
S31508000A6C1A6059680D4A0A405A601A6822F084724C
S31508000A7C22F480321A601A6822F480221A605A68A4
S31508000A8C22F4FE025A604FF41F029A60044B4FF090
S31508000A9C00629A60704700BF001002400000FFF821
S31508000AAC00ED00E0014B1880704700BF5C04002085
S31508000ABC08B500F01BFC0E4B1B6898420FD30D4B68
S31508000ACC1B786BB90B4B01221A700B4B20221A613F
S31508000ADC00F00CFC094B1B881844054B186008BD24
S31508000AEC044B00221A70044B20225A61F0E700BF0F
S31508000AFC600400205E040020000801405C0400200D
S31508000B0C014B20225A6170470008014008B5054B75
S31508000B1C9B6813F4005F01D1002008BDFFF7F0FFB6
S31508000B2C0120FAE70010014008B56420FFF7BAFF68
S31508000B3C08BD08B5FFF7BCFF08BD000008B5274A75
S31508000B4C136823F0070343F002031360136803F0DA
S31508000B5C0703022B3CD1224B1A6842F480221A60F6
S31508000B6C1A6842F480321A601D4B1B6813F4003F56
S31508000B7CFAD01B4A536823F47C1343F4E8135360E6
S31508000B8C136843F080731360154B1B6813F0007FD2
S31508000B9CFAD0134B5A6822F0F0025A605A6822F4BB
S31508000BACE06242F480625A605A6822F460525A60D3
S31508000BBC5A6822F0030242F002025A60084B5B683C
S31508000BCC03F00C03082BF9D10648FFF773FB08BD95
S31508000BDC6821054800F0A4F8BDE700BF00200240D4
S31508000BEC0010024000A24A049818000808B5FFF73E
S31508000BFC5FFCFFF7A3FF08BD08B5FFF7F7FF00F08A
S31508000C0C9BF800F0A7F8FCE770B58AB02E4B9A69EA
S31508000C1C42F001029A619A6902F001020492049A5E
S31508000C2CDA6942F08052DA61DA6902F0805203928C
S31508000C3C039A9A6942F004029A619A6902F00402CC
S31508000C4C0292029A9A6942F010029A619A6902F023
S31508000C5C10020192019ADA6942F40032DA61DB6910
S31508000C6C03F400330093009B42F2200305930123FF
S31508000C7C06930223079300260896144C05A92046CA
S31508000C8CFFF716FD2023636103F18463059304259E
S31508000C9C069505A90E48FFF70BFD40F2044305938C
S31508000CAC0923069303230793089605A92046FFF7FD
S31508000CBCFFFC40F608030593069505A92046FFF7A1
S31508000CCCF7FC0AB070BD00BF0010024000080140D6
S31508000CDC0010014008B5FFF7FDFB0E48FFF790FC26
S31508000CEC0D48FFF78DFC0D4BDA6922F40032DA61F8
S31508000CFC9A6922F010029A619A6922F004029A61A2
S31508000D0CDA6922F08052DA619A6922F001029A6154
S31508000D1C08BD00BF00100140000801400010024049
S31508000D2C08B500F005F8FCE708B5FFF7FDFE08BDA9
S31508000D3C08B5FFF7FEFE08BD08B500F037FDFFF74E
S31508000D4CF3FF00F0B1FA00F064FD00F04BF800F088
S31508000D5C3DF808BD08B5FFF7EBFF00F0B9FA00F04F
S31508000D6C4DF800F001F808BD08B500F095F8012813
S31508000D7C03D00B4B1B78012B00D008BD00F0B6FA3C
S31508000D8C084B1B68084A1268134403F5FA73984211
S31508000D9CF3D3034B00221A7000F00CFDEDE700BFED
S31508000DAC68040020640400206C04002008B5054B78
S31508000DBC1B78012B00D008BD00F098FA024B18607E
S31508000DCCF9E700BF680400206C04002008B5044B42
S31508000DDC01221A70FFF7EAFFFFF7C6FF08BD00BF2E
S31508000DEC6804002008B500F0C7F900F0B1FA024B08
S31508000DFC00221A7008BD00BF3804002000B583B065
S31508000E0C0DF10701084800F0E1FA012802D003B0F9
S31508000E1C5DF804FB054B00221A709DF80710024872
S31508000E2C00F0CAF9F3E700BF70040020380400206C
S31508000E3C7047000008B5054B1B7813B100F0B4F9E0
S31508000E4C08BDC9B200F0A6FAF8E700BF38040020BE
S31508000E5C074B1B78022B05D0032B05D0012B05D08D
S31508000E6C40207047002070470020704700207047CC
S31508000E7C38040020074B1B78022B05D0032B05D012
S31508000E8C012B05D040207047002070470020704782
S31508000E9C002070473804002008B500F07BF903469B
S31508000EAC00B10123184608BD014B00225A70704741
S31508000EBCB0040020034BFE22DA7018710222A3F844
S31508000ECC44207047B004002010B5054C002323704D
S31508000EDCFFF7EAFFFF23E3700123A4F8443010BDA3
S31508000EECB0040020064BFF22DA7000221A715978DA
S31508000EFC59719A71DA711A720622A3F8442070474E
S31508000F0CB004002008B50020FFF7D4FF08BD000088
S31508000F1C074BFF22DA70074A9A6400221A715A7133
S31508000F2C9A710722C3F807200822A3F844207047B1
S31508000F3CB0040020A0180008044BFF22DA7042689F
S31508000F4C9A640122A3F84420704700BFB00400201D
S31508000F5C08B53120FFF7AEFF08BD000038B5084CC0
S31508000F6CFF23E370002525716571FFF771FFA071EA
S31508000F7CE571257265720723A4F8443038BD00BFA5
S31508000F8CB004002038B5FFF78FFF0E4C01252570ED
S31508000F9CFF23E3701023237100236371FFF758FFB7
S31508000FACA071FFF767FFE071FFF764FFC0F3072036
S31508000FBC20726572A5720823A4F8443000F029FC47
S31508000FCC38BD00BFB004002038B50546FFF740FF12
S31508000FDC6A7890420FD90A4CA16C201D00F00AFCC5
S31508000FECFF23E3706A78A36C1344A3646B7801330C
S31508000FFCA4F8443038BD2220FFF75CFFFAE700BF9F
S3150800100CB004002038B50446FFF722FF63789842EF
S3150800101C11D961680A4DA9646278281D00F0EAFBAB
S3150800102CFF23EB706278AB6C1344AB6463780133C3
S3150800103CA5F8443038BD2220FFF73CFFFAE700BF7D
S3150800104CB0040020F8B50546174600244E1E39B1E3
S3150800105C15F8013B1C44E4B2FFF76AFE3146F5E786
S3150800106C3C600120F8BD000010B5084CFF23E37066
S3150800107CE21D4168A06CFFF7E5FF20710023637140
S3150800108CA3710823A4F8443010BD00BFB004002097
S3150800109C38B505460D4B9C6CFFF7DAFE6A1C411EEB
S315080010AC204600F0BAFB60B1084CFF23E370FFF74B
S315080010BCCFFE0138A36C0344A3640123A4F844307F
S315080010CC38BD3120FFF7F6FEFAE700BFB004002062
S315080010DC10B50446FFF7BCFE01386378984213DD59
S315080010EC114BFF22DA700122A3F84420617879B1FA
S315080010FCA21C0D4B986C00F090FB88B161780A4ADB
S3150800110C936C0B44936410BD2220FFF7D3FEFAE7C9
S3150800111C00F093FB0028F6D13120FFF7CBFEF2E75F
S3150800112C3120FFF7C7FEEEE7B004002008B541688A
S3150800113C074B986C00F075FB30B1054BFF22DA7043
S3150800114C0122A3F8442008BD3120FFF7B3FEFAE7C5
S3150800115CB004002008B500F02DFB034BFF22DA7013
S3150800116C0122A3F8442008BDB004002008B589B2B2
S3150800117CFFF760FE08BD0000054B00221A709A6442
S3150800118C83F84320A3F844209A705A70704700BF1E
S3150800119CB0040020034B1B780BB1012070470020CC
S315080011AC704700BFB0040020024B002283F843208E
S315080011BC704700BFB004002008B50378FF2B23D076
S315080011CC354A1278012A2BD1C93B352B53D8DFE87F
S315080011DC03F04052524F52524C43494652525252C5
S315080011EC52525252525252525252525252525252C5
S315080011FC525252525252525252525252312B282E4B
S3150800120C5252523452373A3DFFF7BCFE224B93F8F2
S3150800121C4330012B33D0204BB3F94410002932DC70
S3150800122C08BDFFF7D1FEF1E7FFF7ECFEEEE7FFF797
S3150800123C83FEEBE7FFF718FFE8E7FFF769FEE5E73C
S3150800124CFFF760FEE2E7FFF74DFEDFE7FFF73CFE30
S3150800125CDCE7FFF71DFFD9E7FFF73AFFD6E7FFF7FD
S3150800126C7DFED3E7FFF762FFD0E7FFF773FFCDE705
S3150800127CFFF76EFECAE72020FFF71CFEC6E7102014
S3150800128CFFF718FEC7E71846012380F843300330EA
S3150800129CFFF76CFFC4E700BFB0040020014B002227
S315080012AC1A60704710E000E008B5FFF7F7FF054B2A
S315080012BC054A5A6000229A6005211960034B1A6088
S315080012CC08BD00BF10E000E03F190100FC04002037
S315080012DC044B1B6813F4803F03D0034A136801338D
S315080012EC1360704710E000E0FC04002008B5FFF717
S315080012FCEFFF014B186808BDFC04002008B5FFF782
S3150800130CF5FF08BD70470000054B1B6813F0200F4E
S3150800131C01D100207047024B5B68037001207047AF
S3150800132C0044004010B5094B5860FFF7DFFF00F189
S3150800133C0A04064B1B6813F0800F05D1FFF7F8FC5F
S3150800134CFFF7D4FFA042F4D910BD00BF00440040FB
S3150800135C10B588B04FF461430193002302930393AD
S3150800136C04930C2205920693094C01A92046FEF714
S3150800137CA7FF236923F490432361636923F02A03A7
S3150800138C6361E36843F40053E36008B010BD00BF23
S3150800139C0044004070B506460D4640290ED828462E
S315080013ACFFF7C0FF0024ABB2A3420CD9FFF7C0FC71
S315080013BC305DFFF7B7FF0134A4B2F4E76F2102489A
S315080013CCFFF7AEFCEBE770BDA818000870B5254B07
S315080013DC1C78BCB92448FFF797FF012801D0204692
S315080013EC70BD214B1B78013BDBB23F2BF7D8FFF7BF
S315080013FC7DFF1E4B18601E4B00221A70194B0122DA
S3150800140C1A70ECE706460D46194B1B78013316483D
S3150800141C1844FFF779FF0446012815D1144B1A789E
S3150800142C0132D2B21A70104B1B789A4201D00024A2
S3150800143CD5E71049304600F0DDF90A4B00221A7040
S3150800144C0B4B1B782B70CAE7FFF750FF074B1B6833
S3150800145C6433984203D90024024B1C70BFE700245E
S3150800146CBDE700BF4105002000050020440500200B
S3150800147C420500200105002008B5C1F3080353B93D
S3150800148C03688B4209D040F8041B4FF4007200F035
S3150800149CB1F9012008BD0020FCE70120FAE72DE987
S315080014ACF0410746FFF7BCF9002400E001347F2C15
S315080014BC14D83E68A30006EB03083B445D68FFF7A7
S315080014CC37FC2A46002341460220FFF701FA38B9B1
S315080014DC56F82430AB42E9D0002402E0012400E09F
S315080014EC0024FFF7B7F92046BDE8F08138B50D465C
S315080014FC0C4B984211D004460B4B994207D1094C18
S3150800150C29462046FFF7B8FF48B1204638BDFFF7F5
S3150800151CC6FF0028F4D10024F7E7044CF0E70024B2
S3150800152CF3E700BF4C070020002000084805002000
S3150800153C2DE9F04106460C4617461D4621F4FF7860
S3150800154C28F001080368B3F1FF3F07D03368434519
S3150800155C0BD13368E41A3444043415E04146FFF7DA
S3150800156C8BFF03460028F1D11FE041463046FFF7B2
S3150800157CBDFF06460028ECD1002316E017F8013B00
S3150800158C04F8013B013D0FD0FFF7D2FB331DE31ADC
S3150800159CB3F5007FF2D308F500713046FFF7A6FFC6
S315080015AC064628B1041DE9E701231846BDE8F08173
S315080015BC0023FAE74FF0FF33024A1360024A13601E
S315080015CC704700BF480500204C07002010B54B1E7D
S315080015DC114C241AA34218D8104B984217D90B1839
S315080015EC013B0D4CA34214D80B46014620F4FF7060
S315080015FC20F001000A4CA04203D00A48FFF798FFD6
S3150800160C04E00948FFF794FF00E0002010BD002015
S3150800161CFCE70020FAE700BFFFFF0108FF1F0008E0
S3150800162C00200008480500204C07002030B587B07C
S3150800163C002305934A1E1F4B1B1A9A4231D820F4D5
S3150800164C7F7323F003031C4A93422ED90A18013AD6
S3150800165C184CA2422BD8C01A0144C1F38F25C1F3EA
S3150800166C090109B10135ADB2002401940393012394
S3150800167C0493FFF7D5F8A5420DD9FFF759FB05A931
S3150800168C01A8FFF797F950B9039B03F580630393F9
S3150800169C0134A4B2EFE70124FFF7DCF802E00024DA
S315080016ACFAE70024204607B030BD0024FAE70024E8
S315080016BCF8E700BFFFFF0108FF1F0008104B1B6867
S315080016CCB3F1FF3F19D000B583B00D4A5368916842
S315080016DC0B44D1680B4411690B4451690B4491694D
S315080016EC0B44D26913445B42019301AA04210548B1
S315080016FCFFF76CFF03B05DF804FB0120704700BFD1
S3150800170C4C0700200C2100080D4B1B680D4A12686B
S3150800171C1A440D4B1B6813440C4A126813440C4AA2
S3150800172C12681A440B4B1B681A440B4B1B68134460
S3150800173C0A4A1268DA4201D0002070470120704725
S3150800174C0020000804200008082000080C200008C7
S3150800175C1020000814200008182000080C21000886
S3150800176C08B50E4B1B68B3F1FF3F07D10C4B1B6832
S3150800177CB3F1FF3F09D10123184608BD0748FFF707
S3150800178C8EFE03460028F1D1F6E70548FFF787FEDB
S3150800179C03460028F0D00123EEE700BF4C070020D3
S315080017AC48050020004870470020000808B500F0DE
S315080017BC4FF808BD10B500F038F800B910BDFFF7A2
S315080017CCA5F90028FAD0FFF733FBFFF767FDFEF7FC
S315080017DC39FE00F02EF820F0604020F07F00044B14
S315080017EC986000F026F8446800F034F8A047E5E75E
S315080017FC00ED00E070B50D460446531E9EB23AB194
S3150800180C15F8013B04F8013BFFF792FA3246F4E768
S3150800181C70BD08B5FFF7CEFE08BD08B5FFF7D6FEB6
S3150800182C08BD08B5FFF702FF08BD08B5FFF76CFF42
S3150800183C08BD08B5FFF7B6FF08BD08B5FFF73EFFAC
S3150800184C034608B9184608BDFFF78AFF0346F9E7A9
S3150800185C72B6704762B67047F8B500BFF8BC08BCDC
S3150800186C9E467047F8B500BFF8BC08BC9E46704744
S3150800187C0000002000000000000000000102030424
S3150800188C0607080900000000010203046D61696E71
S3150800189C2E6300004F70656E424C54002E2E2F2E70
S315080018AC2E2F2E2E2F536F757263652F41524D4373
S315080018BC4D335F53544D333246312F7273323332B4
S309080018CC2E63000079
S30D080018D095010008310100082A
S309080018D80D010008E8
S315080018DC00000000EC02002054030020BC0300208A
S315080018EC00000000000000000000000000000000DE
S315080018FC00000000000000000000000000000000CE
S3150800190C00000000000000000000000000000000BD
S3150800191C00000000000000000000000000000000AD
S3150800192C000000000000000000000000000000009D
S3150800193C000000000000000000000000000000008D
S3150800194C000000000000000000000000000000007D
S3150800195C000000000000000000000000000000006D
S3150800196C000000000000000000000000000000005D
S3150800197C000000000000000001000000000000004C
S3150800198C0E33CDAB34126DE6ECDE05000B00000011
S3150800199C000000000000000000000000000000002D
S315080019AC000000000000000000000000000000001D
S315080019BC000000000000000000000000000000000D
S315080019CC00000000000000000000000000000000FD
S31508001CFC0000000000000000500900200100000050
S31108001D0C100000000024F4000400000091
S705080002757B
